 RT2501USB

 Timestamp is 45c1f5e3 (Thu Feb 01 22:14:59 2007)

 Preferred load address is 10000000

 Start         Length     Name                   Class
 0001:00000000 0000094cH .rdata                  CODE
 0001:0000094c 00000066H .rdata$debug            CODE
 0001:000009c0 000254f7H .text                   CODE
 0001:00025eb8 0000003cH .idata$2                CODE
 0001:00025ef4 00000014H .idata$3                CODE
 0001:00025f08 000000ecH .idata$4                CODE
 0001:00025ff4 000003acH .idata$6                CODE
 0001:000263a0 0000009eH .edata                  CODE
 0002:00000000 000000ecH .idata$5                DATA
 0002:000000f0 0000587eH .data                   DATA
 0002:00005980 00001418H .bss                    DATA

  Address         Publics by Value              Rva+Base     Lib:Object

 0000:00000000       ___safe_se_handler_table   00000000     <absolute>
 0000:00000000       ___safe_se_handler_count   00000000     <absolute>
 0001:0000001c       ??_C@_0N@BOOJCAPA@HW?5Diversity?$AA@ 1000101c     mlme.obj
 0001:0000002c       ??_C@_05LKLMIBEG@Ant?9B?$AA@ 1000102c     mlme.obj
 0001:00000034       ??_C@_05JBJBNCIF@Ant?9A?$AA@ 10001034     mlme.obj
 0001:0000003c       ??_C@_0N@ENCHDJIJ@SW?5Diversity?$AA@ 1000103c     mlme.obj
 0001:0000004c       ??_C@_0DC@DNIOBKKO@4?9way?5handshake?5IE?5diff?5among?5As@ 1000104c     mlme.obj
 0001:00000080       ??_C@_0CE@ODBDOOLB@2?9way?5?$CIgroup?5key?$CJ?5handshake?5time@ 10001080     mlme.obj
 0001:000000a4       ??_C@_0BI@IFDLABDB@4?9way?5handshake?5timeout?$AA@ 100010a4     mlme.obj
 0001:000000bc       ??_C@_09CJDAIAGP@MIC?5error?$AA@ 100010bc     mlme.obj
 0001:000000c8       ??_C@_0L@LCBPMDKI@invalid?5IE?$AA@ 100010c8     mlme.obj
 0001:000000d4       ??_C@_0CD@EMJAOFKL@require?5auth?5before?5assoc?1re?9ass@ 100010d4     mlme.obj
 0001:000000f8       ??_C@_0O@IBGJFIPI@class?53?5error?$AA@ 100010f8     mlme.obj
 0001:00000108       ??_C@_0O@ENMDFIGG@class?52?5error?$AA@ 10001108     mlme.obj
 0001:00000118       ??_C@_0CE@IOCPNGNK@AP?5unable?5to?5hanle?5all?5associati@ 10001118     mlme.obj
 0001:0000013c       ??_C@_0BM@OBHJDPBG@DIS?9ASSOC?5due?5to?5inactivity?$AA@ 1000113c     mlme.obj
 0001:00000158       ??_C@_0BK@BAGFOGKD@STA?5is?5leaving?5?1?5has?5left?$AA@ 10001158     mlme.obj
 0001:00000174       ??_C@_0BO@PEBKGJDA@Previous?5Auth?5no?5longer?5valid?$AA@ 10001174     mlme.obj
 0001:00000194       ??_C@_0BD@PBGFPAEA@Unspecified?5Reason?$AA@ 10001194     mlme.obj
 0001:000001a8       ??_C@_08NKCLJDKG@Reserved?$AA@ 100011a8     mlme.obj
 0001:000001b4       ??_C@_19DICJPJO@?$AAT?$AAE?$AAS?$AAT?$AA?$AA@ 100011b4     rtmp_init.obj
 0001:000001c0       ??_C@_1BG@IINBLCLB@?$AAD?$AAt?$AAi?$AAm?$AAP?$AAe?$AAr?$AAi?$AAo?$AAd?$AA?$AA@ 100011c0     rtmp_init.obj
 0001:000001d8       ??_C@_1CE@PCANMBOM@?$AAA?$AAu?$AAt?$AAo?$AAC?$AAh?$AAa?$AAn?$AAn?$AAe?$AAl?$AAS?$AAe?$AAl?$AAe?$AAc?$AAt?$AA?$AA@ 100011d8     rtmp_init.obj
 0001:000001fc       ??_C@_1BC@GBGBNBCD@?$AAC?$AAL?$AAF?$AAa?$AAc?$AAt?$AAo?$AAr?$AA?$AA@ 100011fc     rtmp_init.obj
 0001:00000210       ??_C@_1BC@EGPLFCEP@?$AAN?$AAH?$AAF?$AAa?$AAc?$AAt?$AAo?$AAr?$AA?$AA@ 10001210     rtmp_init.obj
 0001:00000224       ??_C@_1BI@GKAHDKBF@?$AAC?$AAC?$AAX?$AA2?$AAC?$AAo?$AAn?$AAt?$AAr?$AAo?$AAl?$AA?$AA@ 10001224     rtmp_init.obj
 0001:0000023c       ??_C@_1O@LPLILBCD@?$AAP?$AAS?$AAM?$AAo?$AAd?$AAe?$AA?$AA@ 1000123c     rtmp_init.obj
 0001:0000024c       ??_C@_1BE@KABNOABI@?$AAA?$AAd?$AAh?$AAo?$AAc?$AAO?$AAf?$AAd?$AAm?$AA?$AA@ 1000124c     rtmp_init.obj
 0001:00000260       ??_C@_1BI@FJLDDKCH@?$AAN?$AAe?$AAt?$AAw?$AAo?$AAr?$AAk?$AAT?$AAy?$AAp?$AAe?$AA?$AA@ 10001260     rtmp_init.obj
 0001:00000278       ??_C@_1BM@EFMHHLJG@?$AAA?$AAu?$AAt?$AAo?$AAR?$AAe?$AAc?$AAo?$AAn?$AAn?$AAe?$AAc?$AAt?$AA?$AA@ 10001278     rtmp_init.obj
 0001:00000294       ??_C@_1BO@MJECKBG@?$AAS?$AAh?$AAo?$AAw?$AAH?$AAi?$AAd?$AAd?$AAe?$AAn?$AAS?$AAS?$AAI?$AAD?$AA?$AA@ 10001294     rtmp_init.obj
 0001:000002b4       ??_C@_1M@HCFAIFML@?$AAR?$AAa?$AAd?$AAi?$AAo?$AA?$AA@ 100012b4     rtmp_init.obj
 0001:000002c0       ??_C@_1BI@HGMLCLKI@?$AAM?$AAu?$AAl?$AAt?$AAi?$AAp?$AAl?$AAe?$AAI?$AAR?$AAP?$AA?$AA@ 100012c0     rtmp_init.obj
 0001:000002d8       ??_C@_1BG@HGDCKNNC@?$AAW?$AAM?$AAM?$AAC?$AAa?$AAp?$AAa?$AAb?$AAl?$AAe?$AA?$AA@ 100012d8     rtmp_init.obj
 0001:000002f0       ??_C@_1BA@FANIFMBI@?$AAT?$AAX?$AAB?$AAu?$AAr?$AAs?$AAt?$AA?$AA@ 100012f0     rtmp_init.obj
 0001:00000300       ??_C@_1BG@BPJAKMMA@?$AAI?$AAE?$AAE?$AAE?$AA8?$AA0?$AA2?$AA1?$AA1?$AAH?$AA?$AA@ 10001300     rtmp_init.obj
 0001:00000318       ??_C@_1CC@CENNGNJ@?$AAF?$AAr?$AAa?$AAm?$AAe?$AAA?$AAg?$AAg?$AAr?$AAe?$AAg?$AAa?$AAt?$AAi?$AAo?$AAn?$AA?$AA@ 10001318     rtmp_init.obj
 0001:0000033c       ??_C@_1BE@CJFJGBPC@?$AAS?$AAh?$AAo?$AAr?$AAt?$AAS?$AAl?$AAo?$AAt?$AA?$AA@ 1000133c     rtmp_init.obj
 0001:00000350       ??_C@_1BK@KPPOILKG@?$AAB?$AAG?$AAP?$AAr?$AAo?$AAt?$AAe?$AAc?$AAt?$AAi?$AAo?$AAn?$AA?$AA@ 10001350     rtmp_init.obj
 0001:0000036c       ??_C@_1BO@HGPPFMIN@?$AAN?$AAe?$AAt?$AAw?$AAo?$AAr?$AAk?$AAA?$AAd?$AAd?$AAr?$AAe?$AAs?$AAs?$AA?$AA@ 1000136c     rtmp_init.obj
 0001:0000038c       ??_C@_1BA@HCLACGFM@?$AAW?$AAE?$AAP?$AAK?$AAe?$AAy?$AA4?$AA?$AA@ 1000138c     rtmp_init.obj
 0001:0000039c       ??_C@_1BA@OPGHBOOF@?$AAW?$AAE?$AAP?$AAK?$AAe?$AAy?$AA3?$AA?$AA@ 1000139c     rtmp_init.obj
 0001:000003ac       ??_C@_1BA@FHNLHJIA@?$AAW?$AAE?$AAP?$AAK?$AAe?$AAy?$AA2?$AA?$AA@ 100013ac     rtmp_init.obj
 0001:000003bc       ??_C@_1BA@EFGONGGO@?$AAW?$AAE?$AAP?$AAK?$AAe?$AAy?$AA1?$AA?$AA@ 100013bc     rtmp_init.obj
 0001:000003cc       ??_C@_1BG@OIMBEMPB@?$AAV?$AAe?$AAn?$AAd?$AAo?$AAr?$AAD?$AAe?$AAs?$AAc?$AA?$AA@ 100013cc     rtmp_init.obj
 0001:000003e4       ??_C@_19KJNOMKCJ@?$AAS?$AAS?$AAI?$AAD?$AA?$AA@ 100013e4     rtmp_init.obj
 0001:000003f0       ??_C@_1BE@HKNKOMJL@?$AAW?$AAE?$AAP?$AAK?$AAe?$AAy?$AAU?$AAs?$AAe?$AA?$AA@ 100013f0     rtmp_init.obj
 0001:00000404       ??_C@_1BG@CLENCLJC@?$AAA?$AAu?$AAt?$AAh?$AAe?$AAn?$AAT?$AAy?$AAp?$AAe?$AA?$AA@ 10001404     rtmp_init.obj
 0001:0000041c       ??_C@_1BG@MHEIMMBG@?$AAE?$AAn?$AAc?$AAr?$AAy?$AAp?$AAt?$AAi?$AAo?$AAn?$AA?$AA@ 1000141c     rtmp_init.obj
 0001:00000434       ??_C@_1BG@CPCOBECG@?$AAF?$AAr?$AAa?$AAg?$AAT?$AAh?$AAr?$AAe?$AAs?$AAh?$AA?$AA@ 10001434     rtmp_init.obj
 0001:0000044c       ??_C@_1BE@NCNOFIOB@?$AAR?$AAt?$AAs?$AAT?$AAh?$AAr?$AAe?$AAs?$AAh?$AA?$AA@ 1000144c     rtmp_init.obj
 0001:00000460       ??_C@_1BA@DLAHBHMC@?$AAC?$AAh?$AAa?$AAn?$AAn?$AAe?$AAl?$AA?$AA@ 10001460     rtmp_init.obj
 0001:00000470       ??_C@_1BK@CMGABJAK@?$AAW?$AAi?$AAr?$AAe?$AAl?$AAe?$AAs?$AAs?$AAM?$AAo?$AAd?$AAe?$AA?$AA@ 10001470     rtmp_init.obj
 0001:0000048c       ??_C@_1CG@FHJPKHBD@?$AAC?$AAo?$AAu?$AAn?$AAt?$AAr?$AAy?$AAR?$AAe?$AAg?$AAi?$AAo?$AAn?$AAA?$AAB?$AAa?$AAn?$AAd?$AA?$AA@ 1000148c     rtmp_init.obj
 0001:000004b4       ??_C@_1BM@PHDEHLBE@?$AAC?$AAo?$AAu?$AAn?$AAt?$AAr?$AAy?$AAR?$AAe?$AAg?$AAi?$AAo?$AAn?$AA?$AA@ 100014b4     rtmp_init.obj
 0001:000004d0       ??_C@_1O@OADBDALB@?$AAO?$AAp?$AAM?$AAo?$AAd?$AAe?$AA?$AA@ 100014d0     rtmp_init.obj
 0001:000004e0       _ccitt_16Table             100014e0     rtmp_init.obj
 0001:000006e0       ??_C@_07BDGAECLF@CKIP128?$AA@ 100016e0     rtmp_init.obj
 0001:000006e8       ??_C@_06HHMNOKIF@CKIP64?$AA@ 100016e8     rtmp_init.obj
 0001:000006f0       ??_C@_03BKNEFOAH@AES?$AA@  100016f0     rtmp_init.obj
 0001:000006f4       ??_C@_04HNKLFFMO@TKIP?$AA@ 100016f4     rtmp_init.obj
 0001:000006fc       ??_C@_06JCFAKCMD@wep128?$AA@ 100016fc     rtmp_init.obj
 0001:00000704       ??_C@_05PJDLFBFB@wep64?$AA@ 10001704     rtmp_init.obj
 0001:0000070c       ??_C@_04CGFJFPFD@none?$AA@ 1000170c     rtmp_init.obj
 0001:00000714       ??_C@_08FDDFGJNM@rt73?4bin?$AA@ 10001714     rtmp_init.obj
 0001:0000071d       ??_C@_00CNPNBAHC@?$AA@     1000171d     connect.obj
 0001:00000920       ??_C@_1BG@NGFFKKHI@?$AAR?$AAT?$AA2?$AA5?$AA0?$AA1?$AAU?$AAS?$AAB?$AA1?$AA?$AA@ 10001920     wince.obj
 0001:00000938       ??_C@_1BE@BMEIGAKF@?$AAR?$AAT?$AA2?$AA5?$AA0?$AA1?$AAU?$AAS?$AAB?$AA?$AA@ 10001938     wince.obj
 0001:000009c0       _MlmeResume                100019c0 f   mlme.obj
 0001:00000a30       _LinkDownExec              10001a30 f   mlme.obj
 0001:00000a60       _MlmeValidateSSID          10001a60 f   mlme.obj
 0001:00000aa0       _MlmeIsVisibleSSID         10001aa0 f   mlme.obj
 0001:00000ae0       _MlmeCalculateChannelQuality 10001ae0 f   mlme.obj
 0001:00000bc0       _MlmeDynamicTxRateSwitching 10001bc0 f   mlme.obj
 0001:000010c0       _MlmeSetPsmBit             100020c0 f   mlme.obj
 0001:00001120       _MlmeSetTxPreamble         10002120 f   mlme.obj
 0001:00001180       _MlmeUpdateTxRates         10002180 f   mlme.obj
 0001:00001750       _BssTableInit              10002750 f   mlme.obj
 0001:00001780       _BssTableSearch            10002780 f   mlme.obj
 0001:000017f0       _BssSsidTableSearch        100027f0 f   mlme.obj
 0001:00001890       _BssTableSearchWithSSID    10002890 f   mlme.obj
 0001:00001960       _BssTableDeleteEntry       10002960 f   mlme.obj
 0001:00001a10       _BssTableSortByRssi        10002a10 f   mlme.obj
 0001:00001ae0       _BssCipherParse            10002ae0 f   mlme.obj
 0001:00001f30       _MgtMacHeaderInit          10002f30 f   mlme.obj
 0001:00001fb0       _MakeOutgoingFrame         10002fb0 f   mlme.obj
 0001:00002000       _MlmeQueueInit             10003000 f   mlme.obj
 0001:00002070       _MlmeRestartStateMachine   10003070 f   mlme.obj
 0001:00002160       _MsgTypeSubst              10003160 f   mlme.obj
 0001:000023b0       _StateMachineInit          100033b0 f   mlme.obj
 0001:00002420       _StateMachineSetAction     10003420 f   mlme.obj
 0001:00002450       _StateMachinePerformAction 10003450 f   mlme.obj
 0001:00002480       _LfsrInit                  10003480 f   mlme.obj
 0001:000024b0       _RandomByte                100034b0 f   mlme.obj
 0001:00002640       _AsicAdjustTxPower         10003640 f   mlme.obj
 0001:00002990       _AsicSleepThenAutoWakeup   10003990 f   mlme.obj
 0001:00002a10       _AsicForceWakeup           10003a10 f   mlme.obj
 0001:00002a50       _AsicSetBssid              10003a50 f   mlme.obj
 0001:00002ab0       _AsicDisableSync           10003ab0 f   mlme.obj
 0001:00002af0       _AsicEnableBssSync         10003af0 f   mlme.obj
 0001:00002b80       _AsicEnableIbssSync        10003b80 f   mlme.obj
 0001:00002ca0       _AsicSetEdcaParm           10003ca0 f   mlme.obj
 0001:00002e80       _AsicSetSlotTime           10003e80 f   mlme.obj
 0001:00002f30       _AsicBbpTuning             10003f30 f   mlme.obj
 0001:00003240       _AsicAddSharedKeyEntry     10004240 f   mlme.obj
 0001:000033d0       _AsicRemoveSharedKeyEntry  100043d0 f   mlme.obj
 0001:00003420       _RTMPCheckRates            10004420 f   mlme.obj
 0001:000034d0       _AsicSetRxAnt              100044d0 f   mlme.obj
 0001:000036a0       _AsicEvaluateSecondaryRxAnt 100046a0 f   mlme.obj
 0001:00003710       _AsicRxAntEvalTimeout      10004710 f   mlme.obj
 0001:00003730       _AsicRxAntEvalAction       10004730 f   mlme.obj
 0001:000037c0       _StaQuickResponeForRateUpExec 100047c0 f   mlme.obj
 0001:000038f0       _RadarDetectionStart       100048f0 f   mlme.obj
 0001:000039f0       _RadarDetectionStop        100049f0 f   mlme.obj
 0001:00003a80       _RadarChannelCheck         10004a80 f   mlme.obj
 0001:00003b40       _MlmeFreeMemory            10004b40 f   mlme.obj
 0001:00003d20       _MlmeAllocateMemory        10004d20 f   mlme.obj
 0001:00003e20       _MlmeInitMemoryHandler     10004e20 f   mlme.obj
 0001:00003ff0       _MlmeHalt                  10004ff0 f   mlme.obj
 0001:000040d0       _MlmeSuspend               100050d0 f   mlme.obj
 0001:000042f0       _MlmeCheckPsmChange        100052f0 f   mlme.obj
 0001:00004360       _MlmeRadioOff              10005360 f   mlme.obj
 0001:00004520       _BssEntrySet               10005520 f   mlme.obj
 0001:000046f0       _BssTableSetEntry          100056f0 f   mlme.obj
 0001:00004850       _BssTableSsidSort          10005850 f   mlme.obj
 0001:00004ae0       _MacAddrRandomBssid        10005ae0 f   mlme.obj
 0001:00004b10       _MlmeEnqueue               10005b10 f   mlme.obj
 0001:00004be0       _AsicAntennaSetting        10005be0 f   mlme.obj
 0001:00004ec0       _AsicAntennaSelect         10005ec0 f   mlme.obj
 0001:00005080       _AsicSwitchChannel         10006080 f   mlme.obj
 0001:00005470       _MlmeRadioOn               10006470 f   mlme.obj
 0001:00005500       _MlmeHandler               10006500 f   mlme.obj
 0001:00005750       _MlmePeriodicExec          10006750 f   mlme.obj
 0001:00005850       _MlmeAutoScan              10006850 f   mlme.obj
 0001:00005880       _MlmeAutoReconnectLastSSID 10006880 f   mlme.obj
 0001:00005900       _MlmeCheckForFastRoaming   10006900 f   mlme.obj
 0001:00005a80       _MlmeEnqueueForRecv        10006a80 f   mlme.obj
 0001:00005b90       _MlmeInit                  10006b90 f   mlme.obj
 0001:00005d30       _STAMlmePeriodicExec       10006d30 f   mlme.obj
 0001:00006430       _AironetMsgAction          10007430 f   aironet.obj
 0001:00006600       _ChannelLoadRequestAction  10007600 f   aironet.obj
 0001:00006750       _NoiseHistRequestAction    10007750 f   aironet.obj
 0001:000068c0       _AironetFinalReportAction  100078c0 f   aironet.obj
 0001:000069f0       _ChannelLoadReportAction   100079f0 f   aironet.obj
 0001:00006ac0       _NoiseHistReportAction     10007ac0 f   aironet.obj
 0001:00006c10       _AironetAddBeaconReport    10007c10 f   aironet.obj
 0001:00006f80       _AironetCreateBeaconReportFromBssTable 10007f80 f   aironet.obj
 0001:00007150       _BeaconRequestAction       10008150 f   aironet.obj
 0001:000073b0       _AironetReportAction       100083b0 f   aironet.obj
 0001:000074e0       _AironetRequestAction      100084e0 f   aironet.obj
 0001:00007590       _AironetStateMachineInit   10008590 f   aironet.obj
 0001:000075e0       _Sniff2BytesFromNdisBuffer 100085e0 f   rtusb_data.obj
 0001:00007680       _RTMPSendPacket            10008680 f   rtusb_data.obj
 0001:000078a0       _RTUSBFreeDescriptorRequest 100088a0 f   rtusb_data.obj
 0001:00007950       _RTUSBRejectPendingPackets 10008950 f   rtusb_data.obj
 0001:000079d0       _RTUSBSuspendMsduTransmission 100089d0 f   rtusb_data.obj
 0001:00007a00       _RTUSBCalcDuration         10008a00 f   rtusb_data.obj
 0001:00007a80       _RTUSBWriteTxDescriptor    10008a80 f   rtusb_data.obj
 0001:00007d50       _TxFrameIsAggregatible     10008d50 f   rtusb_data.obj
 0001:00007d80       _RTUSBCleanUpMLMEWaitQueue 10008d80 f   rtusb_data.obj
 0001:00007e30       _RTMPSearchTupleCache      10008e30 f   rtusb_data.obj
 0001:00007e90       _RTMPUpdateTupleCache      10008e90 f   rtusb_data.obj
 0001:00007fc0       _RTMPApplyPacketFilter     10008fc0 f   rtusb_data.obj
 0001:00008070       _RTMPReportMicError        10009070 f   rtusb_data.obj
 0001:00008140       _RTUSBMlmeHardTransmit     10009140 f   rtusb_data.obj
 0001:00008300       _RTMPSendNullFrame         10009300 f   rtusb_data.obj
 0001:00008430       _RTMPCalcDuration          10009430 f   rtusb_data.obj
 0001:000084b0       _RTMPCheckDHCPFrame        100094b0 f   rtusb_data.obj
 0001:000085b0       _RTUSBDequeueMLMEPacket    100095b0 f   rtusb_data.obj
 0001:00008680       _MiniportMMRequest         10009680 f   rtusb_data.obj
 0001:00008760       _RTMPCheckRxDescriptor     10009760 f   rtusb_data.obj
 0001:000088b0       _RTMPSendRTSCTSFrame       100098b0 f   rtusb_data.obj
 0001:00008ae0       _RTUSBHardTransmit         10009ae0 f   rtusb_data.obj
 0001:00009aa0       _RTUSBRxPacket             1000aaa0 f   rtusb_data.obj
 0001:0000a780       _RTMPDeQueuePacket         1000b780 f   rtusb_data.obj
 0001:0000a950       _RTUSBResumeMsduTransmission 1000b950 f   rtusb_data.obj
 0001:0000a9e0       _RTMPSendPackets           1000b9e0 f   rtusb_data.obj
 0001:0000aac0       _ReleaseAdapter            1000bac0 f   rtmp_init.obj
 0001:0000ace0       _RTMPFreeAdapter           1000bce0 f   rtmp_init.obj
 0001:0000ad20       _RTUSBWriteHWMACAddress    1000bd20 f   rtmp_init.obj
 0001:0000ade0       _NICReadEEPROMParameters   1000bde0 f   rtmp_init.obj
 0001:0000b270       _NICInitializeAsic         1000c270 f   rtmp_init.obj
 0001:0000b3c0       _NICUpdateRawCounters      1000c3c0 f   rtmp_init.obj
 0001:0000b5a0       _RTMPEqualMemory           1000c5a0 f   rtmp_init.obj
 0001:0000b5d0       _RTMPCompareMemory         1000c5d0 f   rtmp_init.obj
 0001:0000b610       _RTMPZeroMemory            1000c610 f   rtmp_init.obj
 0001:0000b630       _RTMPMoveMemory            1000c630 f   rtmp_init.obj
 0001:0000b650       _AtoH                      1000c650 f   rtmp_init.obj
 0001:0000b6d0       _RTMPInitTimer             1000c6d0 f   rtmp_init.obj
 0001:0000b700       _RTMPSetTimer              1000c700 f   rtmp_init.obj
 0001:0000b750       _RTMPCancelTimer           1000c750 f   rtmp_init.obj
 0001:0000b780       _RTMPSetLED                1000c780 f   rtmp_init.obj
 0001:0000b870       _RTMPSetSignalLED          1000c870 f   rtmp_init.obj
 0001:0000b8f0       _RTMPCckBbpTuning          1000c8f0 f   rtmp_init.obj
 0001:0000b980       _RTMPAllocAdapterBlock     1000c980 f   rtmp_init.obj
 0001:0000b9e0       _NICInitTransmit           1000c9e0 f   rtmp_init.obj
 0001:0000bcc0       _NICInitRecv               1000ccc0 f   rtmp_init.obj
 0001:0000bd40       _RTMPInitAdapterBlock      1000cd40 f   rtmp_init.obj
 0001:0000bf20       _NICReadRegParameters      1000cf20 f   rtmp_init.obj
 0001:0000c3c0       _NICInitAsicFromEEPROM     1000d3c0 f   rtmp_init.obj
 0001:0000c540       _NICResetFromError         1000d540 f   rtmp_init.obj
 0001:0000c560       _NICLoadFirmware           1000d560 f   rtmp_init.obj
 0001:0000c800       _UserCfgInit               1000d800 f   rtmp_init.obj
 0001:0000cb10       _RTMPInitialize            1000db10 f   rtmp_main.obj
 0001:0000cdb0       _RTMPCheckForHang          1000ddb0 f   rtmp_main.obj
 0001:0000cdc0       _RTMPHalt                  1000ddc0 f   rtmp_main.obj
 0001:0000cf80       _RTMPReset                 1000df80 f   rtmp_main.obj
 0001:0000cf90       _RTMPTransferData          1000df90 f   rtmp_main.obj
 0001:0000d0a0       _RTMPPnPEventNotify        1000e0a0 f   rtmp_main.obj
 0001:0000d170       _DriverEntry               1000e170 f   rtmp_main.obj
 0001:0000d270       _STASetInformation         1000e270 f   rtmp_info.obj
 0001:0000e430       _RTMPWPAAddKeyProc         1000f430 f   rtmp_info.obj
 0001:0000e710       _RTMPWPARemoveKeyProc      1000f710 f   rtmp_info.obj
 0001:0000e7d0       _RTMPWPARemoveAllKeys      1000f7d0 f   rtmp_info.obj
 0001:0000e800       _RTMPSetPhyMode            1000f800 f   rtmp_info.obj
 0001:0000ea80       _RTMPSetInformation        1000fa80 f   rtmp_info.obj
 0001:0000eee0       _STAQueryInformation       1000fee0 f   rtmp_info.obj
 0001:0000fc60       _RTMPQueryInformation      10010c60 f   rtmp_info.obj
 0001:00011360       _ARCFOUR_INIT              10012360 f   rtmp_wep.obj
 0001:00011460       _ARCFOUR_BYTE              10012460 f   rtmp_wep.obj
 0001:000114b0       _ARCFOUR_DECRYPT           100124b0 f   rtmp_wep.obj
 0001:000114b0       _ARCFOUR_ENCRYPT           100124b0 f   rtmp_wep.obj
 0001:00011530       _RTMP_CALC_FCS32           10012530 f   rtmp_wep.obj
 0001:00011570       _RTMPSetICV                10012570 f   rtmp_wep.obj
 0001:000115a0       _RTMPInitWepEngine         100125a0 f   rtmp_wep.obj
 0001:00011660       _RTMPEncryptData           10012660 f   rtmp_wep.obj
 0001:000116a0       _RTMPDecryptData           100126a0 f   rtmp_wep.obj
 0001:000117c0       _RTMPTkipSetMICKey         100127c0 f   rtmp_tkip.obj
 0001:00011820       _RTMPTkipAppendByte        10012820 f   rtmp_tkip.obj
 0001:000118e0       _RTMPTkipAppend            100128e0 f   rtmp_tkip.obj
 0001:00011910       _RTMPTkipGetMIC            10012910 f   rtmp_tkip.obj
 0001:00011990       _RTMPInitTkipEngine        10012990 f   rtmp_tkip.obj
 0001:000119f0       _RTMPInitMICEngine         100129f0 f   rtmp_tkip.obj
 0001:00011a80       _RTMPTkipCompareMICValue   10012a80 f   rtmp_tkip.obj
 0001:00011b70       _RTMPCalculateMICValue     10012b70 f   rtmp_tkip.obj
 0001:00011ca0       _RTMPTkipMixKey            10012ca0 f   rtmp_tkip.obj
 0001:00012220       _construct_mic_header1     10013220 f   rtmp_tkip.obj
 0001:000122b0       _construct_mic_header2     100132b0 f   rtmp_tkip.obj
 0001:00012380       _construct_mic_iv          10013380 f   rtmp_tkip.obj
 0001:00012410       _aes128k128d               10013410 f   rtmp_tkip.obj
 0001:00012520       _construct_ctr_preload     10013520 f   rtmp_tkip.obj
 0001:000125d0       _RTMPSoftDecryptTKIP       100135d0 f   rtmp_tkip.obj
 0001:00012860       _RTMPSoftDecryptAES        10013860 f   rtmp_tkip.obj
 0001:00012c40       _AssocTimeout              10013c40 f   assoc.obj
 0001:00012c80       _ReassocTimeout            10013c80 f   assoc.obj
 0001:00012cc0       _DisassocTimeout           10013cc0 f   assoc.obj
 0001:00012cf0       _MlmeAssocReqAction        10013cf0 f   assoc.obj
 0001:000134e0       _MlmeReassocReqAction      100144e0 f   assoc.obj
 0001:00013b00       _MlmeDisassocReqAction     10014b00 f   assoc.obj
 0001:00013bf0       _AssocPostProc             10014bf0 f   assoc.obj
 0001:00013d80       _PeerDisassocAction        10014d80 f   assoc.obj
 0001:00013e50       _AssocTimeoutAction        10014e50 f   assoc.obj
 0001:00013e80       _ReassocTimeoutAction      10014e80 f   assoc.obj
 0001:00013eb0       _DisassocTimeoutAction     10014eb0 f   assoc.obj
 0001:00013ee0       _InvalidStateWhenAssoc     10014ee0 f   assoc.obj
 0001:00013f10       _InvalidStateWhenReassoc   10014f10 f   assoc.obj
 0001:00013f40       _InvalidStateWhenDisassociate 10014f40 f   assoc.obj
 0001:00013f70       _SwitchBetweenWepAndCkip   10014f70 f   assoc.obj
 0001:00014170       _PeerAssocRspAction        10015170 f   assoc.obj
 0001:00014300       _PeerReassocRspAction      10015300 f   assoc.obj
 0001:000144a0       _AssocStateMachineInit     100154a0 f   assoc.obj
 0001:00014650       _AuthTimeout               10015650 f   auth.obj
 0001:00014690       _MlmeAuthReqAction         10015690 f   auth.obj
 0001:00014820       _PeerAuthRspAtSeq2Action   10015820 f   auth.obj
 0001:00014aa0       _PeerAuthRspAtSeq4Action   10015aa0 f   auth.obj
 0001:00014b70       _MlmeDeauthReqAction       10015b70 f   auth.obj
 0001:00014c50       _AuthTimeoutAction         10015c50 f   auth.obj
 0001:00014c80       _InvalidStateWhenAuth      10015c80 f   auth.obj
 0001:00014cb0       _AuthStateMachineInit      10015cb0 f   auth.obj
 0001:00014d60       _PeerDeauthAction          10015d60 f   auth_rsp.obj
 0001:00014e10       _AuthRspStateMachineInit   10015e10 f   auth_rsp.obj
 0001:00014e80       _RTMPusecDelay             10015e80 f i sync.obj
 0001:00014ec0       _BeaconTimeout             10015ec0 f   sync.obj
 0001:00014ef0       _ScanTimeout               10015ef0 f   sync.obj
 0001:00014f20       _MlmeJoinReqAction         10015f20 f   sync.obj
 0001:00014fe0       _MlmeStartReqAction        10015fe0 f   sync.obj
 0001:000151d0       _PeerProbeReqAction        100161d0 f   sync.obj
 0001:00015480       _BeaconTimeoutAtJoinAction 10016480 f   sync.obj
 0001:000154b0       _ScanNextChannel           100164b0 f   sync.obj
 0001:00015860       _InvalidStateWhenScan      10016860 f   sync.obj
 0001:00015890       _InvalidStateWhenJoin      10016890 f   sync.obj
 0001:000158c0       _InvalidStateWhenStart     100168c0 f   sync.obj
 0001:000158f0       _EnqueuePsPoll             100168f0 f   sync.obj
 0001:00015910       _EnqueueBeaconFrame        10016910 f   sync.obj
 0001:000159a0       _BuildChannelList          100169a0 f   sync.obj
 0001:00015bc0       _FirstChannel              10016bc0 f   sync.obj
 0001:00015bd0       _NextChannel               10016bd0 f   sync.obj
 0001:00015c10       _ChangeToCellPowerLimit    10016c10 f   sync.obj
 0001:00015ca0       _ConvertToRssi             10016ca0 f   sync.obj
 0001:00015d90       _MlmeScanReqAction         10016d90 f   sync.obj
 0001:00015f40       _PeerBeaconAtScanAction    10016f40 f   sync.obj
 0001:000162b0       _PeerBeaconAtJoinAction    100172b0 f   sync.obj
 0001:000166d0       _PeerBeacon                100176d0 f   sync.obj
 0001:00016eb0       _ScanTimeoutAction         10017eb0 f   sync.obj
 0001:00016f00       _SyncStateMachineInit      10017f00 f   sync.obj
 0001:00017050       _MlmeCntlInit              10018050 f   connect.obj
 0001:00017060       _LinkDown                  10018060 f   connect.obj
 0001:000173a0       _MlmeCntlConfirm           100183a0 f   connect.obj
 0001:000173c0       _ScanParmFill              100183c0 f   connect.obj
 0001:00017400       _DisassocParmFill          10018400 f   connect.obj
 0001:00017420       _ComposePsPoll             10018420 f   connect.obj
 0001:000174a0       _ComposeNullFrame          100184a0 f   connect.obj
 0001:00017510       _MakeIbssBeacon            10018510 f   connect.obj
 0001:000178b0       _CntlOidScanProc           100188b0 f   connect.obj
 0001:000179c0       _CntlOidRTBssidProc        100189c0 f   connect.obj
 0001:00017c80       _CntlWaitAuthProc          10018c80 f   connect.obj
 0001:00017e00       _LinkUp                    10018e00 f   connect.obj
 0001:000181e0       _IterateOnBssTab           100191e0 f   connect.obj
 0001:000183b0       _IterateOnBssTab2          100193b0 f   connect.obj
 0001:00018480       _CntlOidSsidProc           10019480 f   connect.obj
 0001:00018750       _CntlMlmeRoamingProc       10019750 f   connect.obj
 0001:000187a0       _CntlWaitDisassocProc      100197a0 f   connect.obj
 0001:00018840       _CntlWaitJoinProc          10019840 f   connect.obj
 0001:00018960       _CntlWaitStartProc         10019960 f   connect.obj
 0001:00018a00       _CntlWaitAuthProc2         10019a00 f   connect.obj
 0001:00018b20       _CntlWaitAssocProc         10019b20 f   connect.obj
 0001:00018b80       _CntlWaitReassocProc       10019b80 f   connect.obj
 0001:00018c00       _CntlIdleProc              10019c00 f   connect.obj
 0001:00018ce0       _MlmeCntlMachinePerformAction 10019ce0 f   connect.obj
 0001:00018e80       _MlmeScanReqSanity         10019e80 f   sanity.obj
 0001:00018ef0       _MlmeStartReqSanity        10019ef0 f   sanity.obj
 0001:00018f20       _MlmeAssocReqSanity        10019f20 f   sanity.obj
 0001:00018f60       _MlmeAuthReqSanity         10019f60 f   sanity.obj
 0001:00018fb0       _PeerAssocRspSanity        10019fb0 f   sanity.obj
 0001:000193d0       _PeerDisassocSanity        1001a3d0 f   sanity.obj
 0001:000193d0       _PeerDeauthSanity          1001a3d0 f   sanity.obj
 0001:00019400       _PeerAuthSanity            1001a400 f   sanity.obj
 0001:000194b0       _PeerProbeReqSanity        1001a4b0 f   sanity.obj
 0001:00019520       _GetTimBit                 1001a520 f   sanity.obj
 0001:000195e0       _ChannelSanity             1001a5e0 f   sanity.obj
 0001:00019620       _PeerTxTypeInUseSanity     1001a620 f   sanity.obj
 0001:000196b0       _RTMPWPAWepKeySanity       1001a6b0 f   sanity.obj
 0001:00019740       _RTMPRemoveKeySanity       1001a740 f   sanity.obj
 0001:00019810       _PeerBeaconAndProbeRspSanity 1001a810 f   sanity.obj
 0001:00019fe0       _NetworkTypeInUseSanity    1001afe0 f   sanity.obj
 0001:0001a030       _MD5Init                   1001b030 f   md5.obj
 0001:0001a060       _MD5Transform              1001b060 f   md5.obj
 0001:0001a8e0       _SHAInit                   1001b8e0 f   md5.obj
 0001:0001aea0       _SHAUpdate                 1001bea0 f   md5.obj
 0001:0001af60       _SHAFinal                  1001bf60 f   md5.obj
 0001:0001b080       _aes_set_key               1001c080 f   md5.obj
 0001:0001b8e0       _aes_decrypt               1001c8e0 f   md5.obj
 0001:0001ca20       _MD5Update                 1001da20 f   md5.obj
 0001:0001cae0       _MD5Final                  1001dae0 f   md5.obj
 0001:0001cb60       _hmac_md5                  1001db60 f   md5.obj
 0001:0001cd20       _WpaMsgTypeSubst           1001dd20 f   wpa.obj
 0001:0001cd90       _WpaMacHeaderInit          1001dd90 f   wpa.obj
 0001:0001ce20       _WpaHardTransmit           1001de20 f   wpa.obj
 0001:0001d170       _HMAC_SHA1                 1001e170 f   wpa.obj
 0001:0001d2b0       _PRF                       1001e2b0 f   wpa.obj
 0001:0001d370       _CCKMPRF                   1001e370 f   wpa.obj
 0001:0001d410       _WpaCountPTK               1001e410 f   wpa.obj
 0001:0001d710       _GenRandom                 1001e710 f   wpa.obj
 0001:0001d870       _AES_GTK_KEY_UNWRAP        1001e870 f   wpa.obj
 0001:0001d9e0       _WpaPairMsg1Action         1001e9e0 f   wpa.obj
 0001:0001ded0       _WpaPairMsg3Action         1001eed0 f   wpa.obj
 0001:0001e300       _WpaGroupMsg1Action        1001f300 f   wpa.obj
 0001:0001e7a0       _WpaEAPOLKeyAction         1001f7a0 f   wpa.obj
 0001:0001e990       _WpaPskStateMachineInit    1001f990 f   wpa.obj
 0001:0001e9d0       _MD4Init                   1001f9d0 f   md4.obj
 0001:0001ea00       _MD4Transform              1001fa00 f   md4.obj
 0001:0001f050       _MD4Update                 10020050 f   md4.obj
 0001:0001f110       _MD4Final                  10020110 f   md4.obj
 0001:0001f1c0       _LeapMsgTypeSubst          100201c0 f   leap.obj
 0001:0001f1d0       _LeapMacHeaderInit         100201d0 f   leap.obj
 0001:0001f260       _LeapStartAction           10020260 f   leap.obj
 0001:0001f320       _LeapIdentityAction        10020320 f   leap.obj
 0001:0001f470       _LeapNakeResponse          10020470 f   leap.obj
 0001:0001f5a0       _HashPwd                   100205a0 f   leap.obj
 0001:0001f620       _ParityKey                 10020620 f   leap.obj
 0001:0001f6c0       _DesKey                    100206c0 f   leap.obj
 0001:0001fa60       _Des                       10020a60 f   leap.obj
 0001:00020430       _DesEncrypt                10021430 f   leap.obj
 0001:00020490       _LeapNetworkChallengeAction 10021490 f   leap.obj
 0001:00020690       _ProcessSessionKey         10021690 f   leap.obj
 0001:00020740       _RogueApTableInit          10021740 f   leap.obj
 0001:00020770       _RogueApTableSearch        10021770 f   leap.obj
 0001:000207c0       _RogueApTableSetEntry      100217c0 f   leap.obj
 0001:00020840       _RogueApTableDeleteEntry   10021840 f   leap.obj
 0001:000208b0       _LeapAuthTimeout           100218b0 f   leap.obj
 0001:00020940       _LeapSendRogueAPReport     10021940 f   leap.obj
 0001:00020d00       _CCKMAssocRspSanity        10021d00 f   leap.obj
 0001:00021180       _CCXAdjacentAPReport       10022180 f   leap.obj
 0001:00021590       _PeerChallengeResponse     10022590 f   leap.obj
 0001:000215f0       _LeapNetworkChallengeResponse 100225f0 f   leap.obj
 0001:00021740       _LeapEapolKeyAction        10022740 f   leap.obj
 0001:000219b0       _LeapPeerChallengeAction   100229b0 f   leap.obj
 0001:00021bc0       _LeapMachinePerformAction  10022bc0 f   leap.obj
 0001:00021dd0       _CKIP_key_permute          10022dd0 f   rtmp_ckipmic.obj
 0001:00022180       _bitwise_xor               10023180 f   rtmp_tkip.obj
 0001:00022180       _xor_128                   10023180 f   rtmp_ckipmic.obj
 0001:000221f0       _next_key                  100231f0 f   rtmp_ckipmic.obj
 0001:00022320       _byte_sub                  10023320 f   rtmp_ckipmic.obj
 0001:00022380       _shift_row                 10023380 f   rtmp_ckipmic.obj
 0001:000223f0       _mix_column                100233f0 f   rtmp_ckipmic.obj
 0001:00022570       _RTMPAesEncrypt            10023570 f   rtmp_ckipmic.obj
 0001:00022760       _RTMPCkipDecrypt           10023760 f   rtmp_ckipmic.obj
 0001:000228a0       _RTMGetPCkipPK             100238a0 f   rtmp_ckipmic.obj
 0001:00022980       _RTMPMicGetCoefficient     10023980 f   rtmp_ckipmic.obj
 0001:00022a00       _RTMPMicFinal              10023a00 f   rtmp_ckipmic.obj
 0001:00022ac0       _RTMPMicUpdate             10023ac0 f   rtmp_ckipmic.obj
 0001:00022b40       _RTMPCkipInsertCMIC        10023b40 f   rtmp_ckipmic.obj
 0001:00022db0       _RTUSBBulkOutDataPacket    10023db0 f   wince_bulk.obj
 0001:00022ed0       _RTUSBBulkOutDataPacketComplete 10023ed0 f   wince_bulk.obj
 0001:000230d0       _RTUSBBulkOutBeaconComplete 100240d0 f   wince_bulk.obj
 0001:00023110       _RTUSBBulkOutMLMEPacket    10024110 f   wince_bulk.obj
 0001:00023190       _RTUSBBulkOutMLMEPacketComplete 10024190 f   wince_bulk.obj
 0001:00023200       _RTUSBBulkOutPsPollComplete 10024200 f   wince_bulk.obj
 0001:00023240       _TransferNotify            10024240 f   wince_bulk.obj
 0001:00023260       _RTUSBBulkReceive          10024260 f   wince_bulk.obj
 0001:000233a0       _RTUSBCleanUpDataBulkOutQueue 100243a0 f   wince_bulk.obj
 0001:00023460       _RTUSBCleanUpMLMEBulkOutQueue 10024460 f   wince_bulk.obj
 0001:000234d0       _RTUSBCancelPendingBulkInIRP 100244d0 f   wince_bulk.obj
 0001:00023510       _RTUSBCancelPendingBulkOutIRP 10024510 f   wince_bulk.obj
 0001:000235d0       _RTUSBBulkOutBeacon        100245d0 f   wince_bulk.obj
 0001:00023640       _RTUSBBulkOutPsPoll        10024640 f   wince_bulk.obj
 0001:000236a0       _RTUSBKickBulkOut          100246a0 f   wince_bulk.obj
 0001:00023a30       _RTUSBCancelPendingIRPs    10024a30 f   wince_bulk.obj
 0001:00023a50       _RTUSBInitializeCmdQ       10024a50 f   wince_io.obj
 0001:00023a60       _RTUSB_VendorRequest       10024a60 f   wince_io.obj
 0001:00023bd0       _RTUSBCE_ConfigureDevice   10024bd0 f   wince_io.obj
 0001:00023e20       _RTMPShutdown              10024e20 f   rtmp_main.obj
 0001:00023e20       _AsicLockChannel           10024e20 f   mlme.obj
 0001:00023e20       _Drop                      10024e20 f   mlme.obj
 0001:00023e20       _RTUSB_InterfaceStop       10024e20 f   wince_io.obj
 0001:00023e30       _RTUSBFirmwareRun          10024e30 f   wince_io.obj
 0001:00023e50       _RTUSBSetLED               10024e50 f   wince_io.obj
 0001:00023e80       _RTUSBMultiRead            10024e80 f   wince_io.obj
 0001:00023eb0       _RTUSBMultiWrite           10024eb0 f   wince_io.obj
 0001:00023ee0       _RTUSBReadMACRegister      10024ee0 f   wince_io.obj
 0001:00023f10       _RTUSBWriteMACRegister     10024f10 f   wince_io.obj
 0001:00023f40       _RTUSBReadBBPRegister      10024f40 f   wince_io.obj
 0001:00024080       _RTUSBWriteBBPRegister     10025080 f   wince_io.obj
 0001:00024140       _RTUSBWriteRFRegister      10025140 f   wince_io.obj
 0001:000241e0       _RTUSBReadEEPROM           100251e0 f   wince_io.obj
 0001:00024210       _RTUSBWriteEEPROM          10025210 f   wince_io.obj
 0001:00024240       _RTUSBPutToSleep           10025240 f   wince_io.obj
 0001:00024260       _RTUSBWakeUp               10025260 f   wince_io.obj
 0001:00024280       _RTUSBQueryHardWareRegister 10025280 f   wince_io.obj
 0001:00024310       _RTUSBSetHardWareRegister  10025310 f   wince_io.obj
 0001:00024570       _RTUSBCmdThread            10025570 f   wince_io.obj
 0001:000253c0       _RTUSBEnqueueCmdFromNdis   100263c0 f   wince_io.obj
 0001:00025540       _RTUSBEnqueueInternalCmd   10026540 f   wince_io.obj
 0001:00025670       _ClosePipe                 10026670 f   wince.obj
 0001:000256b0       _RemoveDeviceContext       100266b0 f   wince.obj
 0001:00025750       _UsbDeviceNotify           10026750 f   wince.obj
 0001:000257b0       _DllEntry                  100267b0 f   wince.obj
 0001:000257d0       _RTUSBCE_InterfaceStart    100267d0 f   wince.obj
 0001:00025890       _USBInstallDriver          10026890 f   wince.obj
 0001:00025930       _USBUnInstallDriver        10026930 f   wince.obj
 0001:000259c0       _ParseUsbDescriptors       100269c0 f   wince.obj
 0001:00025b40       _RTUSBCE_ResetEvent        10026b40 f   wince.obj
 0001:00025b70       _RTMPCopyUnicodeString     10026b70 f   wince.obj
 0001:00025bf0       _USBDeviceAttach           10026bf0 f   wince.obj
 0001:00025c56       _DeleteCriticalSection     10026c56 f   Coredll:COREDLL.dll
 0001:00025c5c       _InitializeCriticalSection 10026c5c f   Coredll:COREDLL.dll
 0001:00025c62       __allmul                   10026c62 f   Coredll:COREDLL.dll
 0001:00025c68       _EventModify               10026c68 f   Coredll:COREDLL.dll
 0001:00025c6e       _LeaveCriticalSection      10026c6e f   Coredll:COREDLL.dll
 0001:00025c74       _EnterCriticalSection      10026c74 f   Coredll:COREDLL.dll
 0001:00025c7a       _CreateThread              10026c7a f   Coredll:COREDLL.dll
 0001:00025c80       _NdisQueryPacket           10026c80 f   ndis:NDIS.dll
 0001:00025c86       _NdisStallExecution        10026c86 f   ndis:NDIS.dll
 0001:00025c8c       _RegisterClientSettings    10026c8c f   usbd:USBD.dll
 0001:00025c92       _RegisterClientDriverID    10026c92 f   usbd:USBD.dll
 0001:00025c98       _UnRegisterClientDriverID  10026c98 f   usbd:USBD.dll
 0001:00025c9e       _UnRegisterClientSettings  10026c9e f   usbd:USBD.dll
 0001:00025ca4       __ResetEvent               10026ca4 f i usbclient:usbclient.obj
 0001:00025cbf       _CloseTransferHandle       10026cbf f   usbclient:usbclient.obj
 0001:00025cdc       _DefaultTransferComplete   10026cdc f   usbclient:usbclient.obj
 0001:00025d0f       _GetTransferStatus         10026d0f f   usbclient:usbclient.obj
 0001:00025d3f       _IssueVendorTransfer       10026d3f f   usbclient:usbclient.obj
 0001:00025e66       _ResetDefaultEndpoint      10026e66 f   usbclient:usbclient.obj
 0001:00025eb8       __IMPORT_DESCRIPTOR_COREDLL 10026eb8     Coredll:COREDLL.dll
 0001:00025ecc       __IMPORT_DESCRIPTOR_NDIS   10026ecc     ndis:NDIS.dll
 0001:00025ee0       __IMPORT_DESCRIPTOR_USBD   10026ee0     usbd:USBD.dll
 0001:00025ef4       __NULL_IMPORT_DESCRIPTOR   10026ef4     Coredll:COREDLL.dll
 0002:00000000       __imp__DeleteCriticalSection 10028000     Coredll:COREDLL.dll
 0002:00000004       __imp__InitializeCriticalSection 10028004     Coredll:COREDLL.dll
 0002:00000008       __imp__ResumeThread        10028008     Coredll:COREDLL.dll
 0002:0000000c       __imp__CeSetThreadPriority 1002800c     Coredll:COREDLL.dll
 0002:00000010       __imp___allmul             10028010     Coredll:COREDLL.dll
 0002:00000014       __imp__EventModify         10028014     Coredll:COREDLL.dll
 0002:00000018       __imp__WaitForSingleObject 10028018     Coredll:COREDLL.dll
 0002:0000001c       __imp__LeaveCriticalSection 1002801c     Coredll:COREDLL.dll
 0002:00000020       __imp__EnterCriticalSection 10028020     Coredll:COREDLL.dll
 0002:00000024       __imp__SetLastError        10028024     Coredll:COREDLL.dll
 0002:00000028       __imp__Sleep               10028028     Coredll:COREDLL.dll
 0002:0000002c       __imp__CloseHandle         1002802c     Coredll:COREDLL.dll
 0002:00000030       __imp__CreateThread        10028030     Coredll:COREDLL.dll
 0002:00000034       __imp__CreateEventW        10028034     Coredll:COREDLL.dll
 0002:00000038       __imp__DisableThreadLibraryCalls 10028038     Coredll:COREDLL.dll
 0002:0000003c       __imp__GetLastError        1002803c     Coredll:COREDLL.dll
 0002:00000040       \177COREDLL_NULL_THUNK_DATA 10028040     Coredll:COREDLL.dll
 0002:00000044       __imp__NdisAllocateSpinLock 10028044     ndis:NDIS.dll
 0002:00000048       __imp__NdisReleaseSpinLock 10028048     ndis:NDIS.dll
 0002:0000004c       __imp__NdisAcquireSpinLock 1002804c     ndis:NDIS.dll
 0002:00000050       __imp__NdisFreeSpinLock    10028050     ndis:NDIS.dll
 0002:00000054       __imp__NdisFreeMemory      10028054     ndis:NDIS.dll
 0002:00000058       __imp__NdisAllocateMemoryWithTag 10028058     ndis:NDIS.dll
 0002:0000005c       __imp__NdisMSleep          1002805c     ndis:NDIS.dll
 0002:00000060       __imp__NdisGetSystemUpTime 10028060     ndis:NDIS.dll
 0002:00000064       __imp__NdisQueryBuffer     10028064     ndis:NDIS.dll
 0002:00000068       __imp__NdisQueryPacket     10028068     ndis:NDIS.dll
 0002:0000006c       __imp__NdisInterlockedIncrement 1002806c     ndis:NDIS.dll
 0002:00000070       __imp__NdisFreeBufferPool  10028070     ndis:NDIS.dll
 0002:00000074       __imp__NdisFreePacketPool  10028074     ndis:NDIS.dll
 0002:00000078       __imp__NdisMInitializeTimer 10028078     ndis:NDIS.dll
 0002:0000007c       __imp__NdisSetTimer        1002807c     ndis:NDIS.dll
 0002:00000080       __imp__NdisMSetPeriodicTimer 10028080     ndis:NDIS.dll
 0002:00000084       __imp__NdisMCancelTimer    10028084     ndis:NDIS.dll
 0002:00000088       __imp__NdisCloseConfiguration 10028088     ndis:NDIS.dll
 0002:0000008c       __imp__NdisUnicodeStringToAnsiString 1002808c     ndis:NDIS.dll
 0002:00000090       __imp__NdisReadConfiguration 10028090     ndis:NDIS.dll
 0002:00000094       __imp__NdisOpenConfiguration 10028094     ndis:NDIS.dll
 0002:00000098       __imp__NdisCloseFile       10028098     ndis:NDIS.dll
 0002:0000009c       __imp__NdisUnmapFile       1002809c     ndis:NDIS.dll
 0002:000000a0       __imp__NdisMapFile         100280a0     ndis:NDIS.dll
 0002:000000a4       __imp__NdisOpenFile        100280a4     ndis:NDIS.dll
 0002:000000a8       __imp__NdisInitializeString 100280a8     ndis:NDIS.dll
 0002:000000ac       __imp__NdisInterlockedDecrement 100280ac     ndis:NDIS.dll
 0002:000000b0       __imp__NdisMGetDeviceProperty 100280b0     ndis:NDIS.dll
 0002:000000b4       __imp__NdisMSetAttributesEx 100280b4     ndis:NDIS.dll
 0002:000000b8       __imp__NdisTerminateWrapper 100280b8     ndis:NDIS.dll
 0002:000000bc       __imp__NdisMRegisterMiniport 100280bc     ndis:NDIS.dll
 0002:000000c0       __imp__NdisInitializeWrapper 100280c0     ndis:NDIS.dll
 0002:000000c4       __imp__NdisGetCurrentSystemTime 100280c4     ndis:NDIS.dll
 0002:000000c8       __imp__NdisStallExecution  100280c8     ndis:NDIS.dll
 0002:000000cc       __imp__NdisDeregisterAdapter 100280cc     ndis:NDIS.dll
 0002:000000d0       __imp__NdisRegisterAdapter 100280d0     ndis:NDIS.dll
 0002:000000d4       \177NDIS_NULL_THUNK_DATA   100280d4     ndis:NDIS.dll
 0002:000000d8       __imp__RegisterClientDriverID 100280d8     usbd:USBD.dll
 0002:000000dc       __imp__UnRegisterClientDriverID 100280dc     usbd:USBD.dll
 0002:000000e0       __imp__UnRegisterClientSettings 100280e0     usbd:USBD.dll
 0002:000000e4       __imp__RegisterClientSettings 100280e4     usbd:USBD.dll
 0002:000000e8       \177USBD_NULL_THUNK_DATA   100280e8     usbd:USBD.dll
 0002:000000f0       _ReasonString              100280f0     mlme.obj
 0002:00000138       _BasicRateMask             10028138     mlme.obj
 0002:00000168       _BROADCAST_ADDR            10028168     mlme.obj
 0002:00000170       _RssiSafeLevelForTxRate    10028170     mlme.obj
 0002:00000180       _Phy11BNextRateDownward    10028180     mlme.obj
 0002:00000184       _Phy11BNextRateUpward      10028184     mlme.obj
 0002:00000188       _Phy11BGNextRateDownward   10028188     mlme.obj
 0002:00000194       _Phy11BGNextRateUpward     10028194     mlme.obj
 0002:000001a0       _Phy11ANextRateDownward    100281a0     mlme.obj
 0002:000001ac       _Phy11ANextRateUpward      100281ac     mlme.obj
 0002:000001b8       _RateUpPER                 100281b8     mlme.obj
 0002:000001d0       _RateDownPER               100281d0     mlme.obj
 0002:000001e8       _RateIdToMbps              100281e8     mlme.obj
 0002:000001f8       _RateIdTo500Kbps           100281f8     mlme.obj
 0002:00000214       _SupRateIe                 10028214     mlme.obj
 0002:00000215       _ExtRateIe                 10028215     mlme.obj
 0002:00000216       _ErpIe                     10028216     mlme.obj
 0002:00000217       _DsIe                      10028217     mlme.obj
 0002:00000218       _TimIe                     10028218     mlme.obj
 0002:00000219       _WpaIe                     10028219     mlme.obj
 0002:0000021a       _Wpa2Ie                    1002821a     mlme.obj
 0002:0000021b       _IbssIe                    1002821b     mlme.obj
 0002:0000021c       _Ccx2Ie                    1002821c     mlme.obj
 0002:00000220       _SES_OUI                   10028220     mlme.obj
 0002:00000228       _RF2528RegTable            10028228     mlme.obj
 0002:00000340       _RF5226RegTable            10028340     mlme.obj
 0002:00000930       _AntStr                    10028930     mlme.obj
 0002:00000940       _CISCO_OUI                 10028940     aironet.obj
 0002:00000944       _SNAP_802_1H               10028944     rtusb_data.obj
 0002:0000094c       _SNAP_BRIDGE_TUNNEL        1002894c     rtusb_data.obj
 0002:00000954       _SNAP_AIRONET              10028954     rtusb_data.obj
 0002:0000095c       _CKIP_LLC_SNAP             1002895c     rtusb_data.obj
 0002:00000964       _EAPOL_LLC_SNAP            10028964     rtusb_data.obj
 0002:0000096c       _EAPOL                     1002896c     rtusb_data.obj
 0002:00000970       _IPX                       10028970     rtusb_data.obj
 0002:00000974       _APPLE_TALK                10028974     rtusb_data.obj
 0002:00000978       _RateIdToPlcpSignal        10028978     rtusb_data.obj
 0002:00000984       _OfdmSignalToRateId        10028984     rtusb_data.obj
 0002:00000994       _default_cwmin             10028994     rtusb_data.obj
 0002:00000998       _default_cwmax             10028998     rtusb_data.obj
 0002:0000099c       _default_sta_aifsn         1002899c     rtusb_data.obj
 0002:000009a0       _MapUserPriorityToAccessCategory 100289a0     rtusb_data.obj
 0002:000009a8       _BIT8                      100289a8     rtmp_init.obj
 0002:000009b0       _BIT32                     100289b0     rtmp_init.obj
 0002:00000a30       _CipherName                10028a30     rtmp_init.obj
 0002:00000a50       _NICRegTable               10028a50     rtmp_init.obj
 0002:00000ed0       _BBPRegTable               10028ed0     rtmp_init.obj
 0002:00000f08       _MACRegTable               10028f08     rtmp_init.obj
 0002:00000fa0       _FirmwareImage             10028fa0     rtmp_init.obj
 0002:00001600       _Wpa2AuthEncryptPairs      10029600     rtmp_info.obj
 0002:00001670       _STASupportedOids          10029670     rtmp_info.obj
 0002:000018c8       _FCSTAB_32                 100298c8     rtmp_wep.obj
 0002:00001cc8       _WEPKEY                    10029cc8     rtmp_wep.obj
 0002:00001cd8       _Tkip_Sbox_Lower           10029cd8     rtmp_tkip.obj
 0002:000020d8       _Tkip_Sbox_Upper           1002a0d8     rtmp_tkip.obj
 0002:000024d8       _CipherWpaTemplate         1002a4d8     assoc.obj
 0002:000024f0       _CipherWpa2Template        1002a4f0     assoc.obj
 0002:00002508       _Ccx2IeInfo                1002a508     assoc.obj
 0002:00002510       _A_BAND_REGION_0_CHANNEL_LIST 1002a510     sync.obj
 0002:00002520       _A_BAND_REGION_1_CHANNEL_LIST 1002a520     sync.obj
 0002:00002534       _A_BAND_REGION_2_CHANNEL_LIST 1002a534     sync.obj
 0002:0000253c       _A_BAND_REGION_3_CHANNEL_LIST 1002a53c     sync.obj
 0002:00002544       _A_BAND_REGION_4_CHANNEL_LIST 1002a544     sync.obj
 0002:0000254c       _A_BAND_REGION_5_CHANNEL_LIST 1002a54c     sync.obj
 0002:00002550       _A_BAND_REGION_6_CHANNEL_LIST 1002a550     sync.obj
 0002:00002554       _A_BAND_REGION_7_CHANNEL_LIST 1002a554     sync.obj
 0002:0000256c       _CipherSuiteWpaNoneTkip    1002a56c     connect.obj
 0002:00002582       _CipherSuiteWpaNoneTkipLen 1002a582     connect.obj
 0002:00002584       _CipherSuiteWpaNoneAes     1002a584     connect.obj
 0002:0000259a       _CipherSuiteWpaNoneAesLen  1002a59a     connect.obj
 0002:0000259c       _WPA_OUI                   1002a59c     sanity.obj
 0002:000025a0       _RSN_OUI                   1002a5a0     sanity.obj
 0002:000025a4       _WME_INFO_ELEM             1002a5a4     sanity.obj
 0002:000025ac       _WME_PARM_ELEM             1002a5ac     sanity.obj
 0002:000025b4       _Ccx2QosInfo               1002a5b4     sanity.obj
 0002:000025b8       _RALINK_OUI                1002a5b8     sanity.obj
 0002:000025bc       _NIC_VENDOR_DESC           1002a5bc     oem.obj
 0002:000025e0       _NIC_VENDOR_DESC_LEN       1002a5e0     oem.obj
 0002:000025e4       _NIC_VENDOR_DRIVER_VERSION 1002a5e4     oem.obj
 0002:000025e8       _LINKNAME_STRING           1002a5e8     oem.obj
 0002:0000260c       _NTDEVICE_STRING           1002a60c     oem.obj
 0002:00004e54       _CipherWpaPskTkip          1002ce54     wpa.obj
 0002:00004e6c       _CipherWpaPskTkipLen       1002ce6c     wpa.obj
 0002:00004e70       _CipherWpaPskAes           1002ce70     wpa.obj
 0002:00004e88       _CipherWpaPskAesLen        1002ce88     wpa.obj
 0002:00004e8c       _CipherSuiteCiscoCCKM      1002ce8c     wpa.obj
 0002:00004ea4       _CipherSuiteCiscoCCKMLen   1002cea4     wpa.obj
 0002:00004ea8       _CipherSuiteCiscoCCKM24    1002cea8     wpa.obj
 0002:00004ec2       _CipherSuiteCiscoCCKM24Len 1002cec2     wpa.obj
 0002:00004ec4       _CipherSuiteCiscoCCKMTkip  1002cec4     wpa.obj
 0002:00004edc       _CipherSuiteCiscoCCKMTkipLen 1002cedc     wpa.obj
 0002:00004ee0       _CipherSuiteCiscoCCKMTkip24 1002cee0     wpa.obj
 0002:00004efa       _CipherSuiteCiscoCCKMTkip24Len 1002cefa     wpa.obj
 0002:00004efc       _CipherSuiteCCXTkip        1002cefc     wpa.obj
 0002:00004f14       _CipherSuiteCCXTkipLen     1002cf14     wpa.obj
 0002:00004f18       _CCX_LLC_HDR               1002cf18     wpa.obj
 0002:00004f20       _LLC_NORMAL                1002cf20     wpa.obj
 0002:00004f28       _EAPOL_FRAME               1002cf28     wpa.obj
 0002:00004f30       _PADDING                   1002cf30     md4.obj
 0002:00004f70       _EAP_HEADER                1002cf70     leap.obj
 0002:00004f78       _SNAP_LEAP_ROGUEAP_HDR     1002cf78     leap.obj
 0002:00004f80       _Spbox                     1002cf80     leap.obj
 0002:00005780       _pc1                       1002d780     leap.obj
 0002:000057b8       _totrot                    1002d7b8     leap.obj
 0002:000057c8       _pc2                       1002d7c8     leap.obj
 0002:00005818       _SboxTable                 1002d818     rtmp_ckipmic.obj
 0002:00005918       _vvenderid                 1002d918     wince.obj
 0002:00005944       _pproductid                1002d944     wince.obj
 0002:00005980       _ZERO_MAC_ADDR             1002d980     mlme.obj
 0002:00005986       _SsidIe                    1002d986     mlme.obj
 0002:00005988       _ZeroSsid                  1002d988     mlme.obj
 0002:000059a8       _RTDebugLevel              1002d9a8     rtmp_main.obj
 0002:000069b0       _Asmversion                1002e9b0     leap.obj
 0002:000069b8       _GUsbFuncs                 1002e9b8     <common>
 0002:000069bc       _GhDevice                  1002e9bc     <common>
 0002:000069c0       _GUsbInterface             1002e9c0     <common>
 0002:000069e0       _LocalStrings              1002e9e0     <common>

 entry point at        0001:000257b0

 Static symbols

 0001:0001a930       _SHAHashBlock              1001b930 f   md5.obj
